:100000005BC086C474C073C072C071C070C06FC062
:100010006EC06DC06CC0BFC06AC069C068C067C038
:1000200066C065C064C092C094C073C074C076C01E
:100030007BC095C07FC084C098C00600FF0901A1A5
:1000400001150026FF00750895040900B20201C0E1
:1000500004030904180373006B0061006C00730053
:100060006B0069002E00620069007A0018036D00C1
:10007000610041006300630075004D00650074007D
:10008000650072001201100100000008C016DF05B3
:1000900000010102000109022200010100800A0999
:1000A00004000001030000000921010100012216E3
:1000B000000705810308006411241FBECFE5D2E0CC
:1000C000DEBFCDBF10E0A0E6B0E0E8E0FCE002C09B
:1000D00005900D92A636B107D9F711E0A6E6B0E07B
:1000E00001C01D92AC3AB107E1F706D28BC588CFAB
:1000F000FC0110821182128213828091660090E0CE
:1001000001978A309105B8F58D5E9F4F8F939F932D
:1001100008958DB501C08CB581832DC080913401C7
:1001200081838091350126C080916A00818380910E
:100130006B0020C08091B00081838091B1001AC013
:100140008091AE0081838091AF0014C080916000E7
:10015000E3CF809161008183809162000BC0809128
:10016000AC0081838091AD0005C080913201818314
:1001700080913301808384E00895FC018081807642
:10018000803239F48181813011F0893011F48FEFA0
:10019000089580E0089578941F920F920FB60F9201
:1001A0001124EF92FF920F931F932F933F934F933E
:1001B0005F936F937F938F939F93AF93BF93EF93CF
:1001C000FF9394B125B140916000809169008F5FE9
:1001D00080936900853008F40DC1122F00E0892F4B
:1001E00090E0082B192B222717FD2095322F842F02
:1001F00090E06AE070E0ADD48053984FAA2797FD55
:10020000A095BA2FBC01CD01A9019801B4D47B01FE
:100210008C011092690080916700813009F441C01F
:10022000813038F0823009F476C0833009F0E2C0C2
:10023000ACC087B1807E87B9389A81E0809367002F
:10024000ECE6F0E020E030E040E050E08281938195
:1002500081939193A0E0B0E0280F391F4A1F5B1FE4
:1002600080E0EA3AF80791F7D801C7011AE0B6959D
:10027000A795979587951A95D1F791838083A0E0EC
:10028000B0E0280F391F4A1F5B1F75E05695479550
:10029000379527957A95D1F730933501209334011E
:1002A000A9C087B1807E87B987B1856087B982E0B0
:1002B00080936700E2EBF0E020E030E040E050E0C7
:1002C0008281938181939193A0E0B0E0280F391F40
:1002D0004A1F5B1F80E0E03FF80791F7D801C70194
:1002E0006AE0B695A795979587956A95D1F791831A
:1002F0008083A0E0B0E0280F391F4A1F5B1F05E094
:1003000056954795379527950A95D1F730936B0009
:1003100020936A006FC087B1807E87B987B18660FD
:1003200087B983E080936700E2EFF0E020E030E0FF
:1003300040E050E08281938181939193A0E0B0E00E
:10034000280F391F4A1F5B1F81E0E033F80791F740
:10035000D801C7011AE0B695A795979587951A9584
:10036000D1F791838083A0E0B0E0280F391F4A1FA6
:100370005B1F75E056954795379527957A95D1F788
:100380003093B1002093B00035C087B1807E87B92B
:1003900010926700E6E3F1E020E030E040E050E05A
:1003A0008281938181939193A0E0B0E0280F391F5F
:1003B0004A1F5B1F81E0E437F80791F7D801C701B6
:1003C0006AE0B695A795979587956A95D1F7918339
:1003D0008083A0E0B0E0280F391F4A1F5B1F85E033
:1003E00056954795379527958A95D1F73093AF0065
:1003F0002093AE00369AFF91EF91BF91AF919F91FC
:100400008F917F916F915F914F913F912F911F91AC
:100410000F91FF90EF900F900FBE0F901F901895C7
:1004200020913401309135018091610090916200FA
:1004300028173907D0F080916A0090916B008217DD
:10044000930718F5A901481B590BBA0186E0769568
:1004500067958A95E1F72091AC003091AD00CB0112
:10046000820F931F8417950730F48DB5882369F0A8
:1004700081508DBD0895261B370B4217530728F472
:100480008DB58F3F11F08F5F8DBD08952091B00025
:100490003091B10080916100909162002817390776
:1004A000D0F08091AE009091AF008217930718F5BD
:1004B000A901481B590BBA0196E0769567959A9564
:1004C000E1F72091320130913301CB01820F931F6C
:1004D0008417950730F48CB5882369F081508CBD62
:1004E0000895261B370B4217530728F48CB58F3F0E
:1004F00011F08F5F8CBD0895CF93DF932EE088E1DC
:1005000090E00FB6F894A89581BD0FBE21BD8AD0AA
:10051000B89A20E040EA5FE004C0A895CA010197BC
:10052000F1F72150D1F7B898789480E090E03CD36F
:10053000809360008F3F19F488E38093600084E02B
:1005400090E03AD390936200809361008F5F9F4F59
:1005500031F484E893E0909362008093610083EA31
:1005600080BF8FB584608FBD1DBC1CBC8AE087BB7B
:1005700080EC87B986B18F6C86B91C9AC0E4DCE93F
:10058000A8957ED04DDF82DFCE010197F1F7F8CF3D
:10059000FC019081909366008181882309F440C01A
:1005A000933071F0943028F4913081F09230C1F59D
:1005B00014C0973001F19A3049F1943089F503C0A5
:1005C00083818DBD2DC083818CBD2AC063816093E2
:1005D000600080E090E0F5D223C0928180E06381EA
:1005E00070E0682B792B709362006093610084E067
:1005F00090E0F5D215C0928180E0238130E0822B1B
:10060000932B9093AD008093AC000AC0928180E060
:10061000238130E0822B932B90933301809332011E
:1006200081E0089585B7826085BF8BB780648BBFFA
:100630008BE4809382018AE58093810108951F9362
:10064000DC01162F8091810184FF07C08091820117
:1006500098E889278093820103C08AE5809381010D
:10066000912FE3E8F1E08D9181939150E1F783E8D8
:1006700091E0612F49D11C5F109381011F91089572
:100680001F93CF93DF9360919201635067FDBDC0CC
:1006900080918F01CCE0D0E0C81BD109CA56DE4F53
:1006A00080918E018D3209F09EC0683009F0ABC098
:1006B00083EC809376018AE5809363001092680052
:1006C0008881807639F0CE0158DD282F8F3F09F4DC
:1006D00079C07FC09A8110927F018981882321F49B
:1006E0001092800122E067C0853019F49093930145
:1006F00061C0863009F04AC08B81813041F484E8C2
:1007000090E0909391018093900122E13BC0823070
:1007100041F486E990E0909391018093900122E268
:1007200031C08330D1F48A81882341F480E590E0A0
:10073000909391018093900124E024C0813019F4BA
:1007400084E590E004C08230E1F48CE690E0909380
:1007500091018093900128E115C0813241F488EA2B
:1007600090E0909391018093900129E00BC0823238
:1007700041F48AE390E0909391018093900126E107
:1007800001C020E080E48093680023C0883021F419
:1007900021E085E991E011C0893019F49093950129
:1007A00009C08A3011F421E006C08B3019F48BE4C3
:1007B0008093820120E08FE791E0909391018093F4
:1007C000900107C0888187FD2E8180E880936800B2
:1007D00006C08F81882319F48E81821708F0822F3A
:1007E0008093640010C08091680087FF0CC0CE0128
:1007F000CFDE8F3F21F48EE18093630004C0882315
:1008000011F010926400109292018091630084FFB5
:1008100058C0809164008F3F09F453C0182F89306D
:1008200008F018E0811B809364008091760198E8BD
:10083000892780937601112391F18091680087FFC9
:1008400008C087E791E0612F53DC182F893098F5B5
:1008500026C0209190013091910186FF0DC0A7E73D
:10086000B1E080E090E0F901E80FF91FE491ED9329
:1008700001961817C1F708C0912FD901E7E7F1E0F9
:100880008D9181939150E1F71150812F90E01F5F7E
:100890000196820F931F909391018093900187E7B7
:1008A00091E0612F31D0612F6C5F6C3041F08FEFA0
:1008B0008093640004C08FEF809364006EE16093C6
:1008C000630094E186B3817431F49150D9F71092AA
:1008D000930110928D01DF91CF911F910895A82F60
:1008E000B92F80E090E041E050EA609530E009C027
:1008F0002D9182279795879510F084279527305E54
:10090000C8F36F5FA8F30895EADF8D939D93089570
:10091000CF93CFB7CF93DF93C395B09BE9F7B09B4D
:100920000BC0B09B09C0B09B07C0B09B05C0B09B7B
:1009300003C0B09B01C08BC06F93C0918F01DD27B6
:10094000CA56DE4F2F9365E5B09B03C02F916F9180
:10095000E6CF0F931F934F9320E040E15F9306B3E0
:10096000017400FB27F93F9350E03BE039C011745C
:1009700040642F77012F5F5F1EC0406816B311746B
:100980002F7752501FC0406406B32F770174D1F106
:100990005F5F00C023C0406216B32F77117491F1DE
:1009A0005F5F00C025C001741027515012F45D5FD5
:1009B0000000115027952C3F16B3C8F6117401277B
:1009C000015027952C3FC8F64227499306B301747E
:1009D00010274F73115027952C3FA8F64695469542
:1009E00016B3117479F00127015027952C3F98F622
:1009F0006B5A60F3315006B3B0F600C010E41ABF72
:100A0000002719C03B503195C31BD04010E41ABFDA
:100A10000881033C09F10B34F9F020918D01198113
:100A2000110F1213EDCF4A81441F093651F10D32D7
:100A300011F0013E29F7009394013F915F914F918E
:100A40001F910F912F916F91CAB7C6FD65CFDF91AE
:100A5000CF91CFBFCF91189520919401222369F3B4
:100A600010919201112391F5343092F1309392015B
:100A700020938E0110918F013BE0311B30938F0149
:100A800027C00091920101300CF50AE54F7049F43E
:100A90003091630034FD1DC000936300C6E7D1E0D0
:100AA0001CC03091810134FD14C000938101C2E863
:100AB000D1E013C0052710E000C0000008BB1AC039
:100AC000052710E0221F1DC010E021C04AE502C02A
:100AD00032ED432FC4E1D0E032E017B31164C09A85
:100AE00008B317BB51E420E865E320FF052708BBE6
:100AF000279517951C3FF0F66695B8F7B1F720FFDC
:100B0000052708BB279517951C3FD0F62795179505
:100B100017FF052700001C3F08BBB0F629913A9546
:100B200019F70E7B10919301110FC651D04008BBED
:100B300011F010938D0110E41ABF016017B31E7BF2
:100B4000402F4E7B54E05A95F1F708BB17BB48BBCA
:100B500074CF5527002480FF02C0060E571F660F72
:100B6000771F6115710521F096958795009799F784
:100B7000952F802D0895FF27EE27BB27AA2760FF1A
:100B800004C0A20FB31FE41FF51F220F331F441F21
:100B9000551F969587957795679589F700977607FE
:100BA00071F7CF01BD010895E199FECF9FBB8EBBC8
:100BB000E09A99278DB30895A8E1B0E042E050E0B3
:100BC00013C0262FE199FECF1CBA9FBB8EBB2DBB55
:100BD0000FB6F894E29AE19A0FBE01960895F1DFFC
:100BE000272FF0CFDC01CB01FC01E199FECF06C03D
:100BF000FFBBEEBBE09A31960DB20D9241505040D2
:080C0000B8F70895F894FFCF46
:060C08003484035AFF00D2
:00000001FF
